:04000000B8012C2AED
:100008000800A4003C0884003A086B21841300050A
:100018002C1C3A06031923282408031D1B282A0828
:10002800FF3E031C242864309B212A082428240A24
:10003800FF3003192328240B23282B082428AD0973
:10004800AD0C272ABA006B2184133230A600003089
:10005800A7000B22A00AA50AA201A30100083A05DD
:10006800A600640000083A05A700260627053A06F8
:100078000319A20A0319A30A2708A600A40303194F
:10008800A5030319A00B35282208272AB816B81E7D
:10009800B812B8195328B8158C2003187A280830D4
:1000A800A300A020A20DA30B5528B81E8520AA20C6
:1000B800A620B81A7A207F2022080310272AB8160B
:1000C800B81EB81238196D28FE39B9003815031052
:1000D800272A381A7528A60038168C2003187A287B
:1000E8002608932003187A28B81E272A8520AA20D4
:1000F80038113812B8113C0884003A088417800473
:100108008B283C0884003A0980058417800508007C
:100118007F20AA208520A6203908B8190138A20016
:100128000830A300A20D03187F20031C8520AA20F5
:10013800A620A30B96287F20AA203C0884003A0812
:100148000005FF3E3D0884003B0988283D088400DF
:100158003B088228A501A400B9172730A300103056
:10016800C1200330A300E830C120A3016430C120BE
:10017800A3010A30C1202408CC28A2002508A10028
:100188002408A000EF212008031DB913B91B08009B
:10019800303EA70086120612061283168612061231
:1001A8000612F030860583122708B818F9283A3065
:1001B800A1009830A9213330A6000E211330A100E8
:1001C8008830A9210E216430A8210E216430A8218D
:1001D8002230A6000E212830F8200C30F8200630F6
:1001E800F820B8142708F9283814A600381C07295D
:1001F8000612033C031C0C290C210730A100D03047
:10020800A921031408003814FE3C0319272A0616EE
:10021800A60E381C38108616F030860526080F39C9
:1002280086048612A60E38180E29C830A821031491
:100238000800BA006E21200821040319272A212268
:1002480084133A088006640029292A29A00A031978
:10025800A10F27298006272AA6003C088400093018
:10026800A70003103C21A60CA70B362903143C2930
:100278008413B91D4B2900083A04391D3A06800039
:10028800841700083A04031C3A068000562900081F
:100298003A04031C3A0639193A06800084173A09C9
:1002A80080055629390D0639A0005F21A100A00A52
:1002B8005F210000A92901308A0020088207013443
:1002C80075340334153400343C340C34D934841771
:1002D8008004272AFF3A84178005272AA000A00D4A
:1002E800A00D200D3839C1389F000130A100F4302D
:1002F800A9211F151F197E291E08A10083161E0893
:10030800272A03178D0083168C130C1483120C08EC
:10031800272A03178C0083168C130C1555308D0073
:10032800AA308D008C148C1897290C11272AA30148
:10033800A200FF30A207031CA307031C272A0330CF
:10034800A100DF30A9219D29A101E83EA000A10953
:10035800FC30031CB229A0070318AF29A0076400CA
:10036800A10FAF292018B829A01CBC290000BC295E
:100378000800A101A301A2000230D429A200033081
:10038800D429A101A301A2000130D429A20006307A
:10039800D429A101A301A2000430D429A200053068
:1003A800A80023082102031DDB29220820020430AB
:1003B80003180130031902302805031DFF30272ACE
:1003C8000038031DFF300405031DFF30272A0404ED
:1003D800031DFF30272AA501A4011030A600210D16
:1003E800A40DA50D2208A4022308031C230FA502AF
:1003F8000318052A2208A40723080318230FA507B2
:100408000310A00DA10DA60BF3292008272A1030F0
:10041800A800A101A001A70CA60C031C192A2208F8
:10042800A00723080318230FA107A10CA00CA50CF3
:10043800A40CA80B0F2A2408272AA009A109A00A9E
:100448000319A10A08008313031383126400080028
:100458008316FF308500C0308600D23087008312B3
:10046800850186018701C1309F00831682309F0075
:10047800873081008312C201C3010716871507144C
:10048800E4016430E3004130E9001E30D400D501B6
:100498000230BE00BF01E830D2000330D300E8309C
:1004A800D6000330D700C801C901E8017F30E20057
:1004B80000308A018521D30001308A018521D200CC
:1004C80002308A018521D70003308A018521D600B0
:1004D80004308A018521BE00BF0105308A018521CB
:1004E800D400D50106308A018521E40007308A014D
:1004F8008521E10008308A018521E00009308A0160
:100508008521E5008B168B178A110A12902A8B1BFE
:1005180008008A150A16612F64308A019B21003071
:10052800051A0130A00000308A01BD21B200003058
:10053800061B0130A00001308A01BD21B400320839
:10054800840034088A01E421B400B5000030861B19
:100558000130A00001308A01BD21B60036088400B0
:10056800340835048A01E4218A150A12031D202C57
:100578000030051A0130A00001308A01BD21B20007
:100588000030061B0130A00001308A01BD21B400F3
:100598003208840034088A01E421B400B500003030
:1005A800861B0130A00000308A01BD21B600360844
:1005B8008400340835048A01E4218A110A12031DD3
:1005C8005C2F0030051A0130A00000308A01BD21DF
:1005D800B2000030061B0130A00000308A01BD21A6
:1005E800B4003208840034088A01E421B400B5005C
:1005F8000030861B0130A00001308A01BD21B60001
:1006080036088400340835048A01E4218A110A1264
:10061800031D782B0030051A0130A00000308A0134
:10062800BD21B2000030061B0130A00001308A0154
:10063800BD21B4003208840034088A01E421B400E2
:10064800B5000030861B0130A00000308A01BD21B2
:10065800B60036088400340835048A01E4218A117A
:100668000A12031D6A2DFE308A01CD2001308A014D
:10067800CD20FE308A01CD2002308A01CD205430B1
:100688008A01CD2041308A01CD2047308A01CD2012
:100698004C308A01CD2049308A01CD2041308A0171
:1006A800CD2045308A01CD2052308A01CD204230FC
:1006B8008A01CD2041308A01CD2020308A01CD2009
:1006C80056308A01CD2033308A01CD202E308A0160
:1006D800CD2030308A01CD200730A300D0308A01E8
:1006E8009C218A150A164B28FE308A01CD2001303C
:1006F8008A01CD20FE308A01CD2002308A01CD202A
:1007080053308A01CD2045308A01CD2054308A01EA
:10071800CD2055308A01CD2050308A01CD205F3060
:100728008A01CD2031308A01CD2064308A019B2195
:100738000030051A0130A00000308A01BD21B20046
:100748000030061B0130A00000308A01BD21B40032
:100758003208840034088A01EB21B400B500003067
:10076800861B0130A00000308A01BD21B600360882
:10077800340435048A110A12031D782BFE308A01CD
:10078800CD2001308A01CD20FE308A01CD200230F3
:100798008A01CD2053308A01CD2065308A01CD20D1
:1007A80074308A01CD2020308A01CD2069308A0139
:1007B800CD206E308A01CD2064308A01CD20693089
:1007C8008A01CD2072308A01CD2069308A01CD207E
:1007D8007A308A01CD207A308A01CD206F308A01A3
:1007E800CD20FE308A01CD20C0308A01CD20533083
:1007F8008A01CD2052308A01CD2046308A01CD2091
:1008080030308A01CD2032308A01CD2020308A0153
:10081800CD2053308A01CD2058308A01CD20203098
:100828008A01CD207E308A01CD200730A300D03048
:100838008A019C21FE308A01CD2001308A01CD2019
:10084800FE308A01CD2002308A01CD2043308A0152
:10085800CD206F308A01CD206C308A01CD206C30DC
:100868008A01CD2065308A01CD2067308A01CD20EC
:1008780061308A01CD2072308A01CD2065308A012D
:10088800CD2020308A01CD2073308A01CD206F30F1
:100898008A01CD206C308A01CD206F308A01CD20AD
:1008A800FE308A01CD20C0308A01CD2053308A0124
:1008B800CD2052308A01CD2046308A01CD203030FB
:1008C8008A01CD2032308A01CD2020308A01CD2006
:1008D80053308A01CD2058308A01CD2020308A013A
:1008E800CD207E308A01CD200730A300D0308A0188
:1008F8009C21FE308A01CD2001308A01CD20FE30B6
:100908008A01CD2002308A01CD2050308A01CD20C5
:1009180055308A01CD2070308A01CD2020308A01DF
:10092800CD203D308A01CD2020308A01CD205330A2
:100938008A01CD2065308A01CD2074308A01CD200E
:10094800FE308A01CD20C0308A01CD2050308A0186
:10095800CD2045308A01CD206E308A01CD2020304F
:100968008A01CD203D308A01CD2020308A01CD205A
:1009780045308A01CD2078308A01CD2069308A013E
:10098800CD2074308A01CD2064008A110A12061B1A
:10099800602DE030EA000730BC001030BA000730A4
:1009A800BD000830BB006A088A01652000308A0152
:1009B8006520A0308A0163200730BC001030BA00DF
:1009C8000730BD000830BB006A088A016520003086
:1009D8008A016520AA308A0163200730BC001030E4
:1009E800BA000730BD000830BB006A088A016520DC
:1009F80000308A016520A5308A0163200730BC00D9
:100A08001030BA000730BD000830BB006A088A0100
:100A1800652000308A016520F2308A016320FE30AB
:100A28008A01CD2001308A01CD20FE308A01CD20F7
:100A380002308A01CD2049308A01CD206E308A01EA
:100A4800CD2064308A01CD2069308A01CD207230F2
:100A58008A01CD2069308A01CD207A308A01CD20E3
:100A68007A308A01CD206F308A01CD20FE308A018C
:100A7800CD20C0308A01CD2043308A01CD2061309D
:100A88008A01CD206D308A01CD2062308A01CD20C7
:100A980069308A01CD2061308A01CD2074308A0105
:100AA800CD206F308A01CD200730A300D0308A01D5
:100AB8009C218A150A164B28C8308A019B2164009C
:100AC8008A150A16051E4B288A017D2CFE308A01DC
:100AD800CD2001308A01CD20FE308A01CD200230A0
:100AE8008A01CD2053308A01CD2045308A01CD209E
:100AF80054308A01CD2055308A01CD2050308A01EA
:100B0800CD205F308A01CD2032308A01CD2064307B
:100B18008A019B210030051A0130A00000308A01AB
:100B2800BD21B2000030061B0130A00000308A0150
:100B3800BD21B4003208840034088A01EB21B400D6
:100B4800B5000030861B0130A00000308A01BD21AD
:100B5800B6003608340435048A110A12031D6A2DBA
:100B6800FE308A01CD2001308A01CD20FE308A0175
:100B7800CD2002308A01CD2053308A01CD20653046
:100B88008A01CD2074308A01CD2020308A01CD2001
:100B980069308A01CD206E308A01CD2064308A0107
:100BA800CD2069308A01CD2072308A01CD2069308C
:100BB8008A01CD207A308A01CD207A308A01CD2071
:100BC8006F308A01CD20FE308A01CD20C0308A01E5
:100BD800CD2053308A01CD2052308A01CD204630B5
:100BE8008A01CD2030308A01CD2032308A01CD20D3
:100BF80020308A01CD2044308A01CD2058308A0126
:100C0800CD2020308A01CD207E308A01CD200730CA
:100C1800A300D0308A019C21FE308A01CD2001300A
:100C28008A01CD20FE308A01CD2002308A01CD20F4
:100C380043308A01CD206F308A01CD206C308A0183
:100C4800CD206C308A01CD2065308A01CD206730F7
:100C58008A01CD2061308A01CD2072308A01CD20F1
:100C680065308A01CD2020308A01CD2073308A0179
:100C7800CD206F308A01CD206C308A01CD206F30B5
:100C88008A01CD20FE308A01CD20C0308A01CD20D6
:100C980053308A01CD2052308A01CD2046308A0156
:100CA800CD2030308A01CD2032308A01CD2020304D
:100CB8008A01CD2044308A01CD2058308A01CD20C8
:100CC80020308A01CD207E308A01CD200730A30054
:100CD800D0308A019C21FE308A01CD2001308A0162
:100CE800CD20FE308A01CD2002308A01CD2050303F
:100CF8008A01CD2055308A01CD2070308A01CD205F
:100D080020308A01CD203D308A01CD2020308A0153
:100D1800CD2053308A01CD2065308A01CD20743032
:100D28008A01CD20FE308A01CD20C0308A01CD2035
:100D380050308A01CD2045308A01CD206E308A019D
:100D4800CD2020308A01CD203D308A01CD202030B1
:100D58008A01CD2045308A01CD2078308A01CD2006
:100D680069308A01CD2074308A01CD2064008A114F
:100D78000A12061B522FF230EA000730BC0010306E
:100D8800BA000730BD000830BB006A088A01652038
:100D980000308A016520A0308A0163200730BC003A
:100DA8001030BA000730BD000830BB006A088A015D
:100DB800652000308A016520AA308A016320073047
:100DC800BC001030BA000730BD000830BB006A080C
:100DD8008A01652000308A016520A5308A016320D8
:100DE8000730BC001030BA000730BD000830BB0027
:100DF8006A088A01652000308A016520E0308A018E
:100E08006320FE308A01CD2001308A01CD20FE30DA
:100E18008A01CD2002308A01CD2049308A01CD20B7
:100E28006E308A01CD2064308A01CD2069308A0174
:100E3800CD2072308A01CD2069308A01CD207A30E8
:100E48008A01CD207A308A01CD206F308A01CD20E9
:100E5800FE308A01CD20C0308A01CD2043308A017E
:100E6800CD2061308A01CD206D308A01CD206230DD
:100E78008A01CD2069308A01CD2061308A01CD20D8
:100E880074308A01CD206F308A01CD200730A3004D
:100E9800D0308A019C218A150A164B28C8308A014D
:100EA8009B2164008A150A16051E4B288A016F2E9D
:100EB800FE308A01CD2001308A01CD20FE308A0122
:100EC800CD2002308A01CD2053308A01CD206530F3
:100ED8008A01CD2074308A01CD2020308A01CD20AE
:100EE80050308A01CD2061308A01CD2072308A01CC
:100EF800CD2061308A01CD206D308A01CD2065304A
:100F08008A01CD2074308A01CD2072308A01CD202B
:100F180069308A01CD2064308A019B210030051A8E
:100F28000130A00000308A01BD21B2000030061B4C
:100F38000130A00000308A01BD21B40032088400CD
:100F480034088A01EB21B400B5000030861B01305B
:100F5800A00000308A01BD21B600360834043504EB
:100F68008A110A12031D5C2FFE308A01CD20013040
:100F78008A01CD20FE308A01CD2002308A01CD20A1
:100F880054308A01CD206D308A01CD2070308A011D
:100F9800CD2020308A01CD2072308A01CD206530E5
:100FA8008A01CD2074308A01CD2072308A01CD208B
:100FB8006F308A01CD206D308A01CD2061308A01E1
:100FC800CD2072308A01CD2063308A01CD2069306E
:100FD8008A01CD2061308A01CD207E308A01CD2062
:100FE800FE308A01CD20C0308A01CD205308A500EB
:100FF80052088A01AF206D308A01CD2073308A01F2
:10100800CD2065308A01CD2063308A01CD2006309D
:10101800BC004030BA00AC01FF30AA00AB0101307F
:10102800AD005C088A010520DC008A150A12031845
:101038003A280630BC008030BA00AC01FF30AA0064
:10104800AB010130AD005C088A010520DC008A157F
:101058000A1203184D2864008A150A12051A37283F
:101068008A150A1261288A150A120B285208A0004C
:101078005308A1000B30A300B8308A01C2218A1599
:101088000A12031D4B286430D2070318D30A8A01B9
:10109800B82F5208A0005308A100A30164308A01A8
:1010A800CA218A150A12031D5F286430D202003053
:1010B800031C013ED3028A01B82FFE308A01CD20DD
:1010C80001308A01CD20FE308A01CD2002308A010C
:1010D800CD2054308A01CD2065308A01CD206D3075
:1010E8008A01CD2070308A01CD206F308A01CD2051
:1010F80020308A01CD2076308A01CD2069308A01DE
:10110800CD2072308A01CD2061308A01CD20743023
:101118008A01CD2061308A01CD2020308A01CD207E
:1011280020308A01CD207E308A01CD20FE308A0110
:10113800CD20C0308A01CD205708A50056088A0165
:10114800AF206D308A01CD2073308A01CD20653003
:101158008A01CD2063308A01CD2064308A019B2129
:1011680064008A150A12051ABC288A150A12B128C1
:101178000630BC004030BA00AC01FF30AA00AB0119
:101188000130AD005C088A010520DC008A150A12CE
:101198000318EB280630BC008030BA00AC01FF30E1
:1011A800AA00AB010130AD005C088A010520DC0013
:1011B8008A150A120318FF2864008A150A12051AEC
:1011C800E8288A150A1214298A150A12BC28560812
:1011D800A0005708A1000B30A300B8308A01C22133
:1011E8008A150A12031DFC286430D6070318D70A8B
:1011F8008A150A1261285608A0005708A100A30101
:1012080064308A01CA218A150A12031D1129643023
:10121800D6020030031C013ED7028A150A12612843
:10122800FE308A01CD2001308A01CD20FE308A01AE
:10123800CD2002308A01CD2041308A01CD20633093
:101248008A01CD2063308A01CD2065308A01CD2006
:101258006C308A01CD2065308A01CD2072308A0138
:10126800CD2061308A01CD207A308A01CD206930C5
:101278008A01CD206F308A01CD206E308A01CD20C1
:1012880065308A01CD2020308A01CD2020308A01A6
:10129800CD207E308A01CD20FE308A01CD20C0309D
:1012A8008A01CD203F08A5003E088A01AF2064309E
:1012B8008A019B2164008A150A12051A66298A1573
:1012C8000A125B290630BC004030BA00AC01FF307E
:1012D800AA00AB010130AD005C088A010520DC00E2
:1012E8008A150A12031895290630BC008030BA0006
:1012F800AC01FF30AA00AB010130AD005C088A01E7
:101308000520DC008A150A120318A72964008A152B
:101318000A12051A92298A150A12BC298A150A1274
:1013280066293E08A0003F08A100A30114308A01E5
:10133800C2218A150A12031DA429BE0A0319BF0A6D
:101348008A150A1214293E08A0003F08A100A3012B
:1013580001308A01CA218A150A12031DB9290130F0
:10136800BE020030031C013EBF028A150A1214296E
:10137800FE308A01CD2001308A01CD20FE308A015D
:10138800CD2002308A01CD2053308A01CD206F3024
:101398008A01CD2067308A01CD206C308A01CD20AA
:1013A80069308A01CD2061308A01CD2020308A0140
:1013B800CD2044308A01CD2069308A01CD20733098
:1013C8008A01CD2074308A01CD2061308A01CD2078
:1013D8006E308A01CD207A308A01CD2061308A01B1
:1013E800CD207E308A01CD20FE308A01CD20C0304C
:1013F8008A01CD205508A50054088A01AF20633022
:101408008A01CD206D308A01CD2064308A019B216C
:1014180064008A150A12051A142A8A150A12092A5A
:101428000630BC004030BA00AC01FF30AA00AB0166
:101438000130AD005C088A010520DC008A150A121B
:101448000318432A0630BC008030BA00AC01FF30D4
:10145800AA00AB010130AD005C088A010520DC0060
:101468008A150A120318552A64008A150A12051AE1
:10147800402A8A150A126A2A8A150A12142A540856
:10148800A0005508A100A30132308A01C2218A15A3
:101498000A12031D522AD40A0319D50A8A150A12F8
:1014A800BC295408A0005508A100A3010A308A01EC
:1014B800CA218A150A12031D672A0130D402003096
:1014C800031C013ED5028A150A12BC29FE308A0186
:1014D800CD2001308A01CD20FE308A01CD20023096
:1014E8008A01CD2043308A01CD206F308A01CD207A
:1014F80072308A01CD2072308A01CD2065308A0190
:10150800CD206E308A01CD2074308A01CD2065301F
:101518008A01CD2020308A01CD204D308A01CD208E
:1015280033308A01CD2020308A01CD206D308A01E8
:10153800CD2069308A01CD206E308A01CD207E30E1
:101548008A01CD206108A000A1016430A200A30196
:101558008A01EF21E7006108A000A1016430A20020
:10156800A3018A01EF212408E600FE308A01CD207C
:10157800C0308A01CD2067088A01AE202C308A014C
:10158800CD2064000A3066028A150A120318CF2A91
:1015980030308A01CD2066088A01AE2041308A01A8
:1015A800CD2020308A01CD2064308A019B2164003F
:1015B8008A150A12051AE32A8A150A12D82A063049
:1015C800BC004030BA00AC01FF30AA00AB010130CA
:1015D800AD005C088A010520DC008A150A12031890
:1015E800122B0630BC008030BA00AC01FF30AA00D4
:1015F800AB010130AD005C088A010520DC008A15CA
:101608000A1203181D2B64008A150A12051A0F2BDB
:101618008A150A12282B8A150A12E32A6400463012
:1016280061028A150A1203181A2BE10A8A150A128E
:101638006A2A6400153061028A150A12031C252BD8
:10164800E1038A150A126A2AFE308A01CD20013088
:101658008A01CD20FE308A01CD2002308A01CD20BA
:1016680043308A01CD206F308A01CD2072308A0143
:10167800CD2072308A01CD2065308A01CD206E30B0
:101688008A01CD2074308A01CD2065308A01CD20B1
:1016980020308A01CD204D308A01CD2033308A0197
:1016A800CD2020308A01CD206D308A01CD206130D7
:1016B8008A01CD2078308A01CD207E308A01CD2064
:1016C8006008A000A1016430A200A3018A01EF21F3
:1016D800E7006008A000A1016430A200A3018A010C
:1016E800EF212408E600FE308A01CD20C0308A01AF
:1016F800CD2067088A01AE202C308A01CD206400F5
:101708000A3066028A150A1203188D2B30308A01B6
:10171800CD2066088A01AE2041308A01CD202030D4
:101728008A01CD2064308A019B2164008A150A123F
:10173800051AA12B8A150A12962B0630BC004030D8
:10174800BA00AC01FF30AA00AB010130AD005C0863
:101758008A010520DC008A150A120318D02B0630EE
:10176800BC008030BA00AC01FF30AA00AB010130E8
:10177800AD005C088A010520DC008A150A120318EE
:10178800DB2B64008A150A12051ACD2B8A150A125A
:10179800E62B8A150A12A12B6400783060028A159C
:1017A8000A120318D82BE00A8A150A12282B64009B
:1017B800513060028A150A12031CE32BE0038A15D4
:1017C8000A12282B03178D01031353088A018D2150
:1017D800031701308D00031352088A018D21031766
:1017E80002308D00031357088A018D210317033037
:1017F8008D00031356088A018D21031704308D00CC
:1018080003133E088A018D21031705308D00031349
:1018180054088A018D21031707308D0003136108CE
:101828008A018D21031708308D00031360088A018F
:101838008D218A150A164B28FE308A01CD200130E9
:101848008A01CD20FE308A01CD2002308A01CD20C8
:1018580054308A01CD2045308A01CD2053308A0189
:10186800CD2054308A01CD2020308A01CD2043304C
:101878008A01CD206F308A01CD206D308A01CD20BC
:1018880070308A01CD206F308A01CD206E308A01F8
:10189800CD2065308A01CD206E308A01CD2074308C
:1018A8008A01CD2069308A01CD2064308A019B21CC
:1018B8000030051A0130A00000308A01BD21B200B5
:1018C8000030061B0130A00000308A01BD21B400A1
:1018D8003208840034088A01EB21B400B5000030D6
:1018E800861B0130A00000308A01BD21B6003608F1
:1018F800340435048A150A12031D202C02308A018B
:101908007221D8002108D9005808A0005908A10060
:101918000530A200A3018A01EF21D8002108D900CF
:101928005808A0005908A1000A30A200A3018A01A2
:10193800EF21E7005808A0005908A1000A30A200CA
:10194800A3018A01EF212408E600FE308A01CD2098
:1019580001308A01CD20FE308A01CD2002308A0173
:10196800CD2056308A01CD2042308A01CD20613009
:101978008A01CD2074308A01CD2020308A01CD2003
:1019880067088A01AE202C308A01CD2066088A01BA
:10199800AE2056308A01CD2020308A01CD20640047
:1019A8008A150A12871EE72C4F308A01CD204E3047
:1019B8008A01CD2020308A01CD2020308A01CD2017
:1019C8007E308A01CD2064008A150A12871AFB2C02
:1019D8004F308A01CD2046308A01CD2046308A0119
:1019E800CD2020308A01CD207E308A01CD200330E1
:1019F8008A017221C4002108C5004408A0004508D6
:101A0800A1000530A200A3018A01EF21C40021082A
:101A1800C5004408A0004508A1006430A200A30145
:101A28008A01EF21E7004408A0004508A1006430BE
:101A3800A200A3018A01EF212408E600FE308A01F2
:101A4800CD20C0308A01CD2049308A01CD206330B5
:101A58008A01CD2020308A01CD2067088A01AE2076
:101A68002C308A01CD2064000A3066028A150A12D9
:101A78000318412D30308A01CD2066088A01AE2036
:101A880041308A01CD2020308A01CD2020308A01C2
:101A9800CD2050308A01CD2061308A01CD206E30B2
:101AA8008A01CD206E308A01CD2065308A01CD2093
:101AB8006C308A01CD2064008A150A12061B652D38
:101AC800871664008A150A12861B6B2D8712C83088
:101AD8008A019B2164008A150A12051A772D87123C
:101AE8008A150A127A2D8A150A12822C64308A0104
:101AF8009B2164008A150A12051E7A2D00308A017E
:101B08007221C8002108C900FE308A01CD200130A9
:101B18008A01CD20FE308A01CD2002308A01CD20F5
:101B28004D308A01CD206D308A01CD206F308A0179
:101B3800CD2074308A01CD206F308A01CD207230DB
:101B48008A01CD2020308A01CD204908A500480807
:101B58008A01AF2064006508003C8A150A12031D3B
:101B6800C42D20308A01CD204F308A01CD20463047
:101B78008A01CD2046308A01CD208A150A12CD2D42
:101B880020308A01CD204F308A01CD204E308A0185
:101B9800CD2064008A150A12061BD42D0130E500F9
:101BA80064008A150A12861BDA2DE50101308A01C4
:101BB8007221CA002108CB000C30A600A7014A08F0
:101BC800A2004B08A3008A010B22B2002508B3002B
:101BD8003208B13CB2003308031C013E213CB3007B
:101BE8003208A0003308A1006630A200A3018A01D0
:101BF800EF21CC002108CD00FE308A01CD20C03075
:101C08008A01CD2054308A01CD2065308A01CD204B
:101C18006D308A01CD2070308A01CD2065308A016F
:101C2800CD2072308A01CD2061308A01CD207430F8
:101C38008A01CD2075308A01CD2072308A01CD20ED
:101C480061308A01CD2020308A01CD204D08A500C1
:101C58004C088A01AF20DF308A01CD2043308A0149
:101C6800CD2020308A01CD2020308A01CD2020309F
:101C78008A01CD207E308A01CD20C8308A019B217F
:101C880064008A150A12051A532E031709308D00AD
:101C9800031365088A018D218A150A12562E8A15A2
:101CA8000A12822D64308A019B2164008A150A1267
:101CB800051E562EFE308A01CD2001308A01CD2026
:101CC800FE308A01CD2002308A01CD2054308A01AD
:101CD800CD2065308A01CD2073308A01CD20743043
:101CE8008A01CD2020308A01CD2042308A01CD20C2
:101CF80057308A01CD2046308A01CD2020308A0114
:101D0800CD2020308A01CD2020308A01CD202030FE
:101D18008A01CD2020308A01CD2020308A01CD20B3
:101D280020308A01CD207E308A01CD206430A20087
:101D3800A3010730840040308A012620C000230810
:101D4800C1004008A0004108A1000330A300E8300A
:101D58008A01CA218A150A12031DD02EFE308A0173
:101D6800CD20C0308A01CD2044308A01CD205830A2
:101D78008A01CD203D308A01CD204F308A01CD2007
:101D88004E308A01CD2020308A01CD2020308A01B2
:101D9800CD208A150A12EB2EFE308A01CD20C030E4
:101DA8008A01CD2044308A01CD2058308A01CD20C7
:101DB8003D308A01CD204F308A01CD2046308A013E
:101DC800CD2046308A01CD2020308A01CD206430D4
:101DD800A200A3010730840080308A012620C000B9
:101DE8002308C1004008A0004108A1000330A30057
:101DF800E8308A01CA218A150A12031D182F5330A8
:101E08008A01CD2058308A01CD203D308A01CD206D
:101E18004F308A01CD204E308A01CD2020308A01F2
:101E2800CD208A150A122A2F53308A01CD20583026
:101E38008A01CD203D308A01CD204F308A01CD2046
:101E480046308A01CD2046308A01CD20C8308A012B
:101E58009B2164008A150A12051E352F8A150A125D
:101E68009A2E64308A019B2164008A150A12051E85
:101E7800352FFE308A01CD2001308A01CD20FE3079
:101E88008A01CD2002308A01CD2054308A01CD202C
:101E980065308A01CD2073308A01CD2074308A01E3
:101EA800CD2020308A01CD204D308A01CD206F30E1
:101EB8008A01CD2074308A01CD202E308A01CD20B0
:101EC80020308A01CD2054308A01CD2072308A0119
:101ED800CD2061308A01CD207A308A01CD202E3084
:101EE8008A01CD20FE308A01CD20C0308A01CD2064
:101EF80050308A01CD2055308A01CD2070308A01BA
:101F0800CD203D308A01CD204D308A01CD2064306E
:101F18008A01CD2078308A01CD2020308A01CD2059
:101F280050308A01CD2044308A01CD2077308A0193
:101F3800CD203D308A01CD204D308A01CD2073302F
:101F48008A01CD2078308A01CD207F30E900003029
:101F5800061B0130A00000308A01BD21B20000300C
:101F6800861B0130A00000308A01BD21B400320870
:101F7800840034088A01E421B400B5006400340800
:101F880035048A110A16031910280730BC000130DD
:101F9800BA000230B90080308A01302102308A014B
:101FA800302102308A013021FE308A01CD200130F3
:101FB8008A01CD20FE308A01CD2002308A01CD2051
:101FC80053308A01CD2065308A01CD2074308A01D2
:101FD800CD2020308A01CD2044308A01CD205330D5
:101FE8008A01CD204D308A01CD2043308A01CD2091
:101FF80020308A01CD204D308A01CD206F308A01F2
:10200800CD2064308A01CD2065308A01CD2003308F
:10201800A300E8308A019C2164008A110A16061B75
:102028009A28FE308A01CD20C0308A01CD204D305B
:102038008A01CD2064308A01CD2078308A01CD20F4
:1020480020308A01CD2061308A01CD2076308A0186
:10205800CD2061308A01CD206E308A01CD207430C8
:102068008A01CD2069308A01CD202E308A01CD2009
:102078002E308A01CD202E308A01CD2020308A01D1
:10208800CD2020308A01CD2020308A01CD20DF01EB
:1020980064005F0869028A110A16031C6F2807305A
:1020A800BC000130BA000230B90080308A0130210A
:1020B80000308A01302107308A0130215F088A0107
:1020C80030213F08A3003E088A019C21DF0A8A11BB
:1020D8000A16031D4C280730A300D0308A019C2122
:1020E8006908DF00640000305F028A110A16031CC9
:1020F8009A280730BC000130BA000230B90080309D
:102108008A01302100308A01302107308A013021CC
:102118005F088A0130213F08A3003E088A019C21FC
:102128000130DF028A110A160318762864008A1122
:102138000A16861B2429FE308A01CD20C0308A0168
:10214800CD204D308A01CD2073308A01CD207830E2
:102158008A01CD2020308A01CD2061308A01CD202E
:1021680076308A01CD2061308A01CD206E308A0117
:10217800CD2074308A01CD2069308A01CD202E30DF
:102188008A01CD202E308A01CD202E308A01CD2023
:1021980020308A01CD2020308A01CD2020308A01CC
:1021A800CD20DF0164005F0869028A110A16031C4A
:1021B800F9280730BC000130BA000230B90080307D
:1021C8008A01302100308A01302104308A0130210F
:1021D8005F088A0130213F08A3003E088A019C213C
:1021E800DF0A8A110A16031DD6280730A300D0304B
:1021F8008A019C216908DF00640000305F028A11AF
:102208000A16031C24290730BC000130BA0002302A
:10221800B90080308A01302100308A013021043031
:102228008A0130215F088A0130213F08A3003E0857
:102238008A019C210130DF028A110A16031800293D
:10224800C8308A019B2164008A110A16051A2F29B1
:102258008A110A1632298A150A123D2F64308A011A
:102268009B2164008A110A16051E3229FE308A0154
:10227800CD2001308A01CD20FE308A01CD200230E8
:102288008A01CD2054308A01CD2065308A01CD20C5
:1022980073308A01CD2074308A01CD2020308A0124
:1022A800CD2053308A01CD2052308A01CD204630CE
:1022B8008A01CD2020308A01CD2044308A01CD20EA
:1022C80058308A01CD20FE308A01CD20C0308A01E5
:1022D800CD2044308A01CD2069308A01CD20733069
:1022E8008A01CD2074308A01CD203D308A01CD206D
:1022F8004308A50042088A01AF2063308A01CD2037
:102308006D308A01CD208A110A166D2664308A0143
:102318009B2164008A110A16051E95298A110A163E
:102328003A2964308A019B2164008A110A16051E25
:102338009529FE308A01CD2001308A01CD20FE305A
:102348008A01CD2002308A01CD2054308A01CD2067
:1023580065308A01CD2073308A01CD2074308A011E
:10236800CD2020308A01CD2053308A01CD20523033
:102378008A01CD2046308A01CD2020308A01CD2027
:1023880053308A01CD2058308A01CD20FE308A0191
:10239800CD20C0308A01CD2044308A01CD2069305B
:1023A8008A01CD2073308A01CD2074308A01CD2076
:1023B8003D308A01CD204308A50042088A01AF209C
:1023C80063308A01CD206D308A01CD208A110A162A
:1023D800CE2664308A019B2164008A110A16051EE4
:1023E800F8298A110A169D2964308A019B21640004
:1023F8008A110A16051EF829FE308A01CD200130FF
:102408008A01CD20FE308A01CD2002308A01CD20FC
:1024180054308A01CD2065308A01CD2073308A017D
:10242800CD2074308A01CD2020308A01CD20533050
:102438008A01CD2065308A01CD206E308A01CD20F9
:1024480073308A01CD206F308A01CD2072308A0125
:10245800CD2065308A01CD2020308A01CD20523030
:102468008A01CD2042308A01CD2064008A110A16E3
:10247800871C772AFE308A01CD20C0308A01CD2002
:1024880052308A01CD2069308A01CD2062308A011C
:10249800CD2061308A01CD206C308A01CD20743086
:1024A8008A01CD2061308A01CD206D308A01CD208E
:1024B80065308A01CD206E308A01CD2074308A01C2
:1024C800CD206F308A01CD203A308A01CD202030CE
:1024D8008A01CD2053308A01CD2049308A01CD2090
:1024E8008A110A16AD2AFE308A01CD20C0308A0131
:1024F800CD2052308A01CD2069308A01CD2062304A
:102508008A01CD2061308A01CD206C308A01CD202E
:1025180074308A01CD2061308A01CD206D308A0166
:10252800CD2065308A01CD206E308A01CD207430EF
:102538008A01CD206F308A01CD203A308A01CD2022
:1025480020308A01CD204E308A01CD204F308A01BB
:10255800CD20C8308A019B2164008A110A16051E05
:10256800B82A8A110A16002A64308A019B2164005D
:102578008A110A16051EB82AFE308A01CD200130BC
:102588008A01CD20FE308A01CD2002308A01CD207B
:1025980057308A01CD2061308A01CD2072308A01FE
:1025A800CD206D308A01CD202D308A01CD205530C7
:1025B8008A01CD2050308A01CD2020308A01CD20DB
:1025C80045308A01CD2053308A01CD2043308A011D
:1025D800CD20FE308A01CD20C0308A01CD20413087
:1025E8008A01CD2074308A01CD2074308A01CD2033
:1025F80065308A01CD206E308A01CD2064308A0191
:10260800CD2065308A01CD2072308A01CD20653019
:102618008A01CD202E308A01CD202E308A01CD208E
:102628002E308A01CD206430E300DF016400513090
:102638005F028A110A160318312B6308A000A10152
:102648000730840004308A011D2164308A019B21EF
:10265800DF0A8A110A16031D1A2B8A018B220430FD
:102668008A017221C6002108C7008A018B22460808
:10267800A0004708A1006430A200A3018A01EF214D
:10268800E7008A018B224608A0004708A1006430B1
:10269800A200A3018A01EF212408E6008A018B2207
:1026A800FE308A01CD2001308A01CD20FE308A011A
:1026B800CD2002308A01CD2049308A01CD20543006
:1026C8008A01CD2061308A01CD2067308A01CD2072
:1026D8006C308A01CD2069308A01CD206F308A01A3
:1026E800CD2020308A01CD2067088A01AE202C3009
:1026F8008A01CD208A018B2264000A3066028A1181
:102708000A1603188A2B30308A01CD208A018B22C1
:1027180066088A01AE2041308A01CD2020308A0126
:10272800CD207E308A01CD208A018B22FE308A019D
:10273800CD20C0308A01CD204D308A01CD203330E4
:102748008A01CD205F308A01CD2056308A01CD2004
:1027580065308A01CD206C308A01CD203D308A0158
:10276800CD2064088A01AE208A018B220030061B26
:102778000130A00000308A01BD21B2006408A00029
:102788001E308A01CD21B4003208840034088A0141
:10279800E421B400B5006400340835048A110A162F
:1027A8000319E02B8A018B22E40A8A018B22643008
:1027B8006407E3008A018B228A018B220030861B82
:1027C8000130A00000308A01BD21B2006408A000D9
:1027D80000308A01C521B4003208840034088A0117
:1027E800E421B400B5006400340835048A110A16DF
:1027F8000319082C8A018B22E4038A018B22643096
:102808006407E3008A018B228A018B2264308A01E3
:102818009B218A018B2264008A110A16051A202C32
:102828006430E300031706308D00031364088A013F
:102838008D218A150A164B288A110A16312BDF01B9
:1028480064005F0869028A110A16031C592C0730B4
:10285800BC000130BA000230B90080308A01302152
:1028680000308A01302107308A0130215F088A014F
:1028780030210730BC000130BA000230B900803086
:102888008A01302100308A01302104308A01302148
:102898005F088A0130213F08A3003E088A019C2175
:1028A800DF0A8A110A16031D242C08006908DF00B4
:1028B800640000305F028A110A16031C922C07304C
:1028C800BC000130BA000230B90080308A013021E2
:1028D80000308A01302107308A0130215F088A01DF
:1028E80030210730BC000130BA000230B900803016
:1028F8008A01302100308A01302104308A013021D8
:102908005F088A0130213F08A3003E088A019C2104
:102918000130DF028A110A1603185C2C0800DF0157
:1029280064005F0862028A110A16031CC92C07306A
:10293800BC000130BA000230B90080308A01302171
:1029480000308A01302106308A0130215F088A016F
:1029580030210730BC000130BA000230B9008030A5
:102968008A01302100308A01302105308A01302166
:102978005F088A0130213F08A3003E088A019C2194
:10298800DF0A8A110A16031D942C5208CE00530838
:10299800CF008A110A16F5256208DF0064000030AE
:1029A8005F028A110A16031C082D0730BC0001308B
:1029B800BA000230B90080308A01302100308A0123
:1029C800302106308A0130215F088A013021073022
:1029D800BC000130BA000230B90080308A013021D1
:1029E80000308A01302105308A0130215F088A01D0
:1029F80030213F08A3003E088A019C210130DF02F4
:102A08008A110A160318D22C0800DF0164005F0837
:102A180062028A110A16031C3F2D0730BC000130E0
:102A2800BA000230B90080308A01302100308A01B2
:102A3800302107308A0130215F088A0130210730B0
:102A4800BC000130BA000230B90080308A01302160
:102A580000308A01302105308A0130215F088A015F
:102A680030213F08A3003E088A019C21DF0A8A1111
:102A78000A16031D0A2D5608CE005708CF008A11E2
:102A88000A16F5256208DF00640000305F028A112B
:102A98000A16031C7E2D0730BC000130BA00023034
:102AA800B90080308A01302100308A013021073096
:102AB8008A0130215F088A0130210730BC000130CB
:102AC800BA000230B90080308A01302100308A0112
:102AD800302105308A0130215F088A0130213F0802
:102AE800A3003E088A019C210130DF028A110A16E0
:102AF8000318482D0800DF0164005F0862028A118C
:102B08000A16031CB52D0730BC000130BA0002308C
:102B1800B90080308A01302100308A013021063026
:102B28008A0130215F088A0130210730BC0001305A
:102B3800BA000230B90080308A01302100308A01A1
:102B4800302104308A0130215F088A0130213F0892
:102B5800A3003E088A019C21DF0A8A110A16031D78
:102B6800802D5608CE005708CF008A110A16F52581
:102B78006208DF00640000305F028A110A16031C35
:102B8800F42D0730BC000130BA000230B9008030A3
:102B98008A01302100308A01302106308A01302133
:102BA8005F088A0130210730BC000130BA000230CA
:102BB800B90080308A01302100308A013021043088
:102BC8008A0130215F088A0130213F08A3003E08AE
:102BD8008A019C210130DF028A110A160318BE2DD2
:102BE8000800DF014E08A0004F08A1006430A200D1
:102BF800A3018A01EF21B2002108B3005F08A000F9
:102C0800A1013308A30032088A01C7218A110A16D4
:102C1800031D6A2E64308A019B216308A000A1016C
:102C28000730840004308A011D210030051A013064
:102C3800A00000308A01BD21B2000030061B01301F
:102C4800A00000308A01BD21B40032088400340895
:102C58008A01EB21B400B5000030861B0130A000CA
:102C680000308A01BD21B6003408350484003608D6
:102C78008A01EB21B600B7006400360837048A11D0
:102C88000A160319652EFE308A01CD2001308A010B
:102C9800CD20FE308A01CD2002308A01CD2053306C
:102CA8008A01CD2054308A01CD204F308A01CD20B1
:102CB80050308A01CD2021308A01CD208A110A1690
:102CC800D12FDF0A8A110A16031DF62D8A018B22DD
:102CD80008008A018B22E030EA008A018B22073043
:102CE800BC001030BA000730BD000830BB006A08CD
:102CF8008A01652000308A01652051308A016320ED
:102D08008A018B226430A200A3010730840040307E
:102D18008A012620C0002308C1008A018B220730BF
:102D2800BC001030BA000730BD000830BB006A088C
:102D38008A01652002308A0165208A014A20DD0067
:102D48008A018B220730BC001030BA000730BD0062
:102D58000830BB006A088A01652003308A016520B3
:102D68008A014A20DE008A018B225D08A600A7019D
:102D7800A2010130A3008A010B22B2002508B3008A
:102D88005E083207C20033080318013EC3008A01F7
:102D98008B2208008A018B22F230EA008A018B22FA
:102DA8000730BC001030BA000730BD000830BB0047
:102DB8006A088A01652000308A01652051308A013D
:102DC80063208A018B226430A200A30107308400AB
:102DD80080308A012620C0002308C1008A018B2286
:102DE8000730BC001030BA000730BD000830BB0007
:102DF8006A088A01652002308A0165208A014A2012
:102E0800DD008A018B220730BC001030BA00073081
:102E1800BD000830BB006A088A01652003308A01BA
:102E280065208A014A20DE008A018B225D08A600FF
:102E3800A701A2010130A3008A010B22B2002508D4
:102E4800B3005E083207C20033080318013EC3000E
:102E58008A018B220800FE308A01CD2001308A01C8
:102E6800CD20FE308A01CD2002308A01CD20563097
:102E78008A01CD2042308A01CD2061308A01CD20DF
:102E880074308A01CD2020308A01CD2062308A0139
:102E9800CD2061308A01CD2073308A01CD20733076
:102EA8008A01CD206F308A01CD20FE308A01CD20E5
:102EB800C0308A01CD2049308A01CD206E308A0188
:102EC800CD2020308A01CD2043308A01CD206130C9
:102ED8008A01CD2072308A01CD2069308A01CD2047
:102EE80063308A01CD2061308A01CD202E308A01DD
:102EF800CD202E308A01CD202E308A01CD208A1196
:102F08000A165A240730BC000130BA000230B90052
:102F180080308A01302100308A01302107308A014F
:102F2800302100308A0130210730BC000130BA005E
:102F38000230B90080308A01302100308A01302106
:102F480004308A01302100308A013021871603308D
:102F5800A300E8308A019C2102308A017221D8003E
:102F68002108D9005808A0005908A1000530A2007E
:102F7800A3018A01EF21D8002108D9005808A00030
:102F88005908A100A30182308A01CF218A110A16AB
:102F9800031DAB2F8A150A16B428FE308A01CD20EE
:102FA800C0308A01CD2050308A01CD2072308A018C
:102FB800CD2065308A01CD206D308A01CD20693061
:102FC8008A01CD2020308A01CD2050308A01CD20C1
:102FD80045308A01CD206E308A01CD200730BC00F3
:102FE8000130BA000230B90080308A013021003047
:102FF8008A01302107308A01302100308A013021CE
:103008000730BC000130BA000230B90080308A01B4
:10301800302100308A01302104308A01302100300B
:103028008A013021871264308A019B210030051AF9
:103038000130A00000308A01BD21B2000030061B1B
:103048000130A00000308A01BD21B400320884009C
:1030580034088A01EB21B400B5000030861B01302A
:10306800A00000308A01BD21B600360834043504BA
:103078008A150A16031D172864308A019B216400EB
:103088008A150A16051E4B288A150A164028643028
:103098008A019B2164008A150A16051E4B28FE30FA
:1030A8008A01CD2001308A01CD20FE308A01CD2051
:1030B80002308A01CD2050308A01CD2072308A0139
:1030C800CD2065308A01CD206D308A01CD20693050
:1030D8008A01CD2020308A01CD2050308A01CD20B0
:1030E80045308A01CD206E308A01CD20FE308A011C
:1030F800CD20C0308A01CD2070308A01CD206530C6
:103108008A01CD2072308A01CD2020308A01CD205D
:1031180069308A01CD206E308A01CD2069308A015C
:10312800CD207A308A01CD2069308A01CD206130E6
:103138008A01CD2072308A01CD2065308A01CD20E8
:1031480064308A019B2164008A150A16051EB4287A
:1031580064008A110A12861F5C2F8A150A16A42891
:10316800FE308A01CD2001308A01CD20FE308A014F
:10317800CD2002308A01CD2041308A01CD20743023
:103188008A01CD2074308A01CD2069308A01CD2092
:1031980076308A01CD2061308A01CD207A308A01CB
:1031A800CD2069308A01CD206F308A01CD206E3064
:1031B8008A01CD2065308A01CD20FE308A01CD20DC
:1031C800C0308A01CD206D308A01CD206F308A0150
:1031D800CD2074308A01CD206F308A01CD20723025
:1031E8008A01CD2065308A01CD2020308A01CD208A
:1031F80074308A01CD2061308A01CD2067308A0180
:10320800CD206C308A01CD2069308A01CD206F3005
:103218008A01CD202E308A01CD202E308A01CD2082
:103228002E308A01CD206430E300DF016400513084
:103238005F028A150A16031831296308A000A10144
:103248000730840004308A011D2164308A019B21E3
:10325800DF0A8A150A16031D1A2964306407E30079
:10326800DF01640015305F028A150A1603184C291D
:103278006308A000A1010730840004308A011D21E1
:1032880064308A019B21DF0A8A150A16031D352935
:103298008A018B22FE308A01CD2001308A01CD209F
:1032A800FE308A01CD2002308A01CD2047308A01C4
:1032B800CD204F308A01CD202E308A01CD202E30EE
:1032C8008A01CD202E308A01CD208A018B224130FF
:1032D800E9008A018B22D001D1018A018B228A114F
:1032E8000A1623248A018B22E8018A018B220030E6
:1032F800051A0130A00000308A01BD21B20000305B
:10330800061B0130A00000308A01BD21B40032083C
:10331800840034088A01EB21B400B5000030861B14
:103328000130A00000308A01BD21B6003408350400
:10333800840036088A01EB21B600B700640036081D
:1033480037048A150A160319CD298A018B22FE3003
:103358008A01CD2001308A01CD20FE308A01CD209E
:1033680002308A01CD2053308A01CD2054308A01A1
:10337800CD204F308A01CD2050308A01CD20213018
:103388008A01CD208A018B228A110A16D12F8A013F
:103398008B228A018B2264008A150A16871C102A40
:1033A8008A018B22FE308A01CD2001308A01CD208E
:1033B800FE308A01CD2002308A01CD2052308A01A8
:1033C800CD2069308A01CD2062308A01CD2061305C
:1033D8008A01CD206C308A01CD2074308A01CD203D
:1033E80061308A01CD206D308A01CD2065308A0197
:1033F800CD206E308A01CD2074308A01CD206F3007
:103408008A01CD2021308A01CD208A018B228A11A0
:103418000A16D12F8A018B228A018B2202308A0157
:103428007221D8002108D9008A018B225808A000EF
:103438005908A1000530A200A3018A01EF21D80094
:103448002108D9008A018B225808A0005908A10038
:10345800A30164308A01CF218A110A16031D2F2F78
:103468008A018B225808A0005908A100A3018730BF
:103478008A01CA218A150A16031D432A87128A015E
:103488008B225808A0005908A100A30182308A01A4
:10349800C2218A150A16031D522A87168A018B2211
:1034A80001308A017221CA002108CB008A018B22CF
:1034B8000C30A600A7014A08A2004B08A3008A0105
:1034C8000B22B2002508B3003208B13CB200330821
:1034D800031C013E213CB3003208A0003308A100C0
:1034E8006630A200A3018A01EF21CC002108CD009B
:1034F8008A018B224C08A0004D08A100A30132309C
:103508008A01CA218A150A16031DC62A8A018B2236
:10351800FE308A01CD20C0308A01CD204D308A018D
:10352800CD2061308A01CD2078308A01CD2020302D
:103538008A01CD2054308A01CD2065308A01CD2002
:103548006D308A01CD2070308A01CD2065308A0126
:10355800CD2072308A01CD2061308A01CD207430AF
:103568008A01CD2075308A01CD2072308A01CD20A4
:1035780061308A01CD208A018B228A110A16D12F47
:103588008A018B228A018B2264000A3068028A151C
:103598000A160318D02AE80A8A018B2200308A0109
:1035A8007221C8002108C9008A018B224808A0009E
:1035B8004908A100A30114308A01CF21B20065088F
:1035C800A00000308A01C521B40032088400340804
:1035D8008A01E421B400B5006808A0000A308A0115
:1035E800BD21B60034083504840036088A01E42178
:1035F800B600B7006400360837048A150A1603199E
:10360800842B8A018B22D00A0319D10A8A018B22C2
:103618005008A0005108A100A30103308A01D2215B
:103628008A150A16031D482B8A018B22FE308A014F
:10363800CD2001308A01CD20FE308A01CD20023014
:103648008A01CD2042308A01CD206C308A01CD20FC
:103658006F308A01CD2063308A01CD2063308A0122
:10366800CD2061308A01CD2074308A01CD206F30A1
:103678008A01CD2021308A01CD208A018B228A112E
:103688000A16D12F8A018B228A018B22FE308A01E9
:10369800CD2001308A01CD20FE308A01CD200230B4
:1036A8008A01CD2041308A01CD206E308A01CD209B
:1036B8006F308A01CD206D308A01CD2061308A01BA
:1036C800CD206C308A01CD2069308A01CD2061304F
:1036D8008A01CD2020308A01CD2052308A01CD20A8
:1036E80055308A01CD204E308A01CD2021308A0103
:1036F800CD208A018B228A150A164D2F8A018B222A
:103708008A018B228A110A166D268A018B224208A9
:10371800A0004308A100A30100308A01C721B2001C
:103728004208A0004308A1005508A30054088A01D4
:10373800CF21B4003208840034088A01E421B4009F
:10374800B5006400340835048A150A160319E62BF7
:103758008A018B22D001D1018A018B22FE308A0195
:10376800CD2001308A01CD20FE308A01CD200230E3
:103778008A01CD204F308A01CD2073308A01CD20B7
:1037880074308A01CD2061308A01CD2063308A01EE
:10379800CD206F308A01CD206C308A01CD206F306A
:1037A8008A01CD2020308A01CD2044308A01CD20E5
:1037B80058308A01CD208A018B228A150A16392FA2
:1037C8008A018B228A018B224008A0004108A100AF
:1037D8000330A300E8308A01CA218A150A16031D9E
:1037E800202C8A018B22D001D1018A018B22FE3044
:1037F8008A01CD2001308A01CD20FE308A01CD20FA
:1038080002308A01CD2042308A01CD2057308A010A
:10381800CD2046308A01CD2020308A01CD20443089
:103828008A01CD2058308A01CD208A018B228A1541
:103838000A16392F8A018B228A018B220030051A39
:103848000130A00000308A01BD21B2000030061B03
:103858000130A00000308A01BD21B4003208840084
:1038680034088A01EB21B400B5000030861B013012
:10387800A00000308A01BD21B60034083504840058
:1038880036088A01EB21B600B70064003608370411
:103898008A150A160319742C8A018B22FE308A01B4
:1038A800CD2001308A01CD20FE308A01CD200230A2
:1038B8008A01CD2053308A01CD2054308A01CD2091
:1038C8004F308A01CD2050308A01CD2021308A0125
:1038D800CD208A018B228A110A16D12F8A018B22C8
:1038E8008A018B228A110A16CE268A018B22420867
:1038F800A0004308A100A30100308A01C721B2003B
:103908004208A0004308A1005508A30054088A01F2
:10391800CF21B4003208840034088A01E421B400BD
:10392800B5006400340835048A150A160319D62C24
:103938008A018B22D001D1018A018B22FE308A01B3
:10394800CD2001308A01CD20FE308A01CD20023001
:103958008A01CD204F308A01CD2073308A01CD20D5
:1039680074308A01CD2061308A01CD2063308A010C
:10397800CD206F308A01CD206C308A01CD206F3088
:103988008A01CD2020308A01CD2053308A01CD20F4
:1039980058308A01CD208A018B228A150A164D2FAC
:1039A8008A018B228A018B220030051A0130A0007F
:1039B80000308A01BD21B2000030061B0130A00092
:1039C80000308A01BD21B4003208840034088A011D
:1039D800EB21B400B5000030861B0130A000003098
:1039E8008A01BD21B60034083504840036088A01EE
:1039F800EB21B600B7006400360837048A150A16AA
:103A080003192A2D8A018B22FE308A01CD2001302C
:103A18008A01CD20FE308A01CD2002308A01CD20D6
:103A280053308A01CD2054308A01CD204F308A018D
:103A3800CD2050308A01CD2021308A01CD208A0145
:103A48008B228A110A16D12F8A018B228A018B2296
:103A58004008A0004108A1000330A300E8308A0113
:103A6800CA218A150A16031D642D8A018B22D001EA
:103A7800D1018A018B22FE308A01CD2001308A01D2
:103A8800CD20FE308A01CD2002308A01CD2042307F
:103A98008A01CD2057308A01CD2046308A01CD20B9
:103AA80020308A01CD2053308A01CD2058308A0138
:103AB800CD208A018B228A150A164D2F8A018B2266
:103AC8008A018B220030051A0130A00000308A01DB
:103AD800BD21B2000030061B0130A00000308A0171
:103AE800BD21B4003208840034088A01EB21B400F7
:103AF800B5000030861B0130A00000308A01BD21CE
:103B0800B60034083504840036088A01EB21B60073
:103B1800B7006400360837048A150A160319B82D49
:103B28008A018B22FE308A01CD2001308A01CD2006
:103B3800FE308A01CD2002308A01CD2053308A011F
:103B4800CD2054308A01CD204F308A01CD2050300D
:103B58008A01CD2021308A01CD208A018B228A1149
:103B68000A16D12F8A018B228A018B2204308A01FE
:103B78007221C6002108C7008A018B224608A000CE
:103B88004708A10060088A01C621B2006908A000A0
:103B980041308A01BD21B4003208840034088A010A
:103BA800E421B400B5006400340835048A150A1607
:103BB80003191D2E8A018B22FE308A01CD20013087
:103BC8008A01CD20FE308A01CD2002308A01CD2025
:103BD80049308A01CD204D308A01CD2033308A0109
:103BE800CD2020308A01CD2065308A01CD20633078
:103BF8008A01CD2063308A01CD2065308A01CD202D
:103C080073308A01CD2073308A01CD2069308A0152
:103C1800CD2076308A01CD2061308A01CD20213037
:103C28008A01CD208A018B228A110A16D12F8A0196
:103C38008B228A018B224608A0004708A100600851
:103C48008A01C621B2006908A00041308A01C52155
:103C5800B4003208840034088A01E421B400B500B5
:103C68006400340835048A150A160319692E8A0176
:103C78008B220230E9028A018B220730BC00013016
:103C8800BA000230B90080308A01302100308A0140
:103C9800302107308A01302169088A0130218A01E0
:103CA8008B220730BC000130BA000230B9008030E6
:103CB8008A01302100308A01302104308A01302104
:103CC80069088A0130218A018B228A018B224608E1
:103CD800A0004708A10061088A01CE21B200690846
:103CE800A0007F308A01CD21B40032088400340856
:103CF8008A01E421B400B5006400340835048A154B
:103D08000A160319B52E8A018B220230E9078A01A7
:103D18008B220730BC000130BA000230B900803075
:103D28008A01302100308A01302107308A01302190
:103D380069088A0130218A018B220730BC000130D2
:103D4800BA000230B90080308A01302100308A017F
:103D5800302104308A01302169088A0130218A0122
:103D68008B228A018B226908A600A7016430A20071
:103D7800A3018A010B22DA002508DB008A018B22C5
:103D88005A08A0005B08A1007F30A200A3018A01A5
:103D9800EF21DA002108DB008A018B225808A000F5
:103DA8005908A1000A30A200A3018A01EF21E70007
:103DB8008A018B225808A0005908A1000A30A200E5
:103DC800A3018A01EF212408E6008A018B22FE3034
:103DD8008A01CD2001308A01CD20FE308A01CD2014
:103DE80002308A01CD2056308A01CD2042308A0126
:103DF800CD2061308A01CD2074308A01CD20203059
:103E08008A01CD2067088A01AE202C308A01CD2096
:103E180066088A01AE2056308A01CD208A018B229D
:103E2800FE308A01CD20C0308A01CD2053308A016E
:103E3800CD2070308A01CD2065308A01CD206530D3
:103E48008A01CD2064308A01CD2020308A01CD201E
:103E58005B08A5005A088A01AF2025308A01CD20C9
:103E68008A018B228A150A1679298A018B228A11DE
:103E78000A165A248A018B228A110A1693248A0167
:103E88008B228A110A1609258A018B228A150A169D
:103E980071298A018B228A110A165A248A018B22D7
:103EA8008A110A1693248A018B228A110A167F2501
:103EB8008A018B228A150A1671296308A000A101BC
:0E3EC8000730840004308A011D210B1109000F
:02400E00393F38
:104200000300E8000300E80002001E0000003C007C
:044210006400000046
:00000001FF
